:100000000C9452000C946F000C946F000C946F00D1
:100010000C946F000C946F000C946F000C946F00A4
:100020000C946F000C946F000C946F000C946F0094
:100030000C946F000C946F000C946F000C946F0084
:100040000C94B4000C946F000C946F000C946F002F
:100050000C946F000C946F000C946F000C946F0064
:100060000C946F000C946F00000000002500280025
:100070002B0000000000240027002A0004040404D0
:100080000404040402020202020203030303030342
:10009000010204081020408001020408102001021F
:1000A0000408102011241FBECFEFD8E0DEBFCDBF63
:1000B00011E0A0E0B1E0E0EAFAE002C005900D92A4
:1000C000A030B107D9F721E0A0E0B1E001C01D9256
:1000D000AD30B207E1F70E94FE000C944E050C947F
:1000E0000000CF93DF9390E0FC01E057FF4F249195
:1000F00084589F4FFC0184918823D1F090E0880FB1
:10010000991FFC01EE58FF4FA591B491FC01E859ED
:10011000FF4FC591D49161110EC09FB7F8948C9197
:10012000E22FE0958E238C932881E223E8839FBF02
:10013000DF91CF9108958FB7F894EC91E22BEC9377
:100140008FBFF6CF8E50806480937C0080917A00C0
:10015000806480937A0080917A0086FDFCCF809144
:1001600078009091790008951F920F920FB60F9228
:1001700011242F933F938F939F93AF93BF938091BD
:10018000090190910A01A0910B01B0910C013091ED
:10019000080123E0230F2D3758F50196A11DB11D4D
:1001A000209308018093090190930A01A0930B0109
:1001B000B0930C018091040190910501A09106017A
:1001C000B09107010196A11DB11D80930401909388
:1001D0000501A0930601B0930701BF91AF919F91D4
:1001E0008F913F912F910F900FBE0F901F901895F8
:1001F00026E8230F0296A11DB11DD2CFCF93DF9326
:1002000000D000D000D01F92CDB7DEB7789484B56F
:10021000826084BD84B5816084BD85B5826085BD02
:1002200085B5816085BD80916E00816080936E0090
:100230001092810080918100826080938100809182
:100240008100816080938100809180008160809333
:1002500080008091B10084608093B1008091B000F3
:1002600081608093B00080917A00846080937A00EE
:1002700080917A00826080937A0080917A00816018
:1002800080937A0080917A00806880937A0010923F
:10029000C10061E08AE00E94710061E08BE00E9491
:1002A000710061E083E00E94710060E081E10E94E2
:1002B000710060E082E10E94710060E08FE00E94C6
:1002C000710060E080E10E94710010928000109245
:1002D000810081EA8093800089E080938100109200
:1002E0008B0010928A001092B0001092B10083EA45
:1002F0008093B00081E08093B1001092B30010921F
:10030000B4002224239460E0A62E60E0B62E8EE096
:100310000E94A20087369105B4F0853321E0920750
:100320000CF4AFC0833032E093070CF4ADC0813DD4
:1003300022E092070CF4ABC08F3993400CF0A9C0B7
:1003400084E0898301C0198281E10E94A2009E831A
:100350008D838FE00E94A200092E000CAA0BBB0B1C
:100360002D813E81A901330F660B770B840F951FFA
:10037000A61FB71F912C812CB7FD0AC04C01811517
:100380009440A105B10524F088248A9453E0952E69
:1003900082E10E94A2009E838D8380E10E94A200E0
:1003A0006C01990FEE08FF082D813E81C901330FC2
:1003B000AA0BBB0B8C0D9D1DAE1DBF1DD12CC12CDE
:1003C000B7FD0AC06C0181159440A105B10524F068
:1003D000CC24CA9443E0D42E3324339481E088168D
:1003E00082E098060CF4312C4424439421E0C21698
:1003F00022E0D2060CF4412CB401092C000C880B2D
:10040000990B0E942C0420E030EC4FE754E40E944A
:1004100082038B018F839D83B6010D2C000C880B0A
:10042000990B0E942C0420E030EC4FE754E40E942A
:1004300082033B017C016A837B828C835F2C398140
:10044000333009F482C038F5313009F462C03230FB
:1004500009F472C000E010E021E0821622E092066A
:100460000CF46EC031E0C31632E0D3060CF4D0C0F9
:100470001F821D82612C712C80E8E82E9FE3F92EEB
:1004800091C021E0298360CF32E039835DCF83E0E2
:1004900058CF25E0F7CF8981843009F472C08530C8
:1004A000C9F681E0881682E098064CF0809102013E
:1004B000811105C08091000182258093000121E017
:1004C000C21622E0D2064CF080910301811105C0D2
:1004D00080910101822580930101309202014092B6
:1004E000030180910001612C712C20E8E22E3FE392
:1004F000F32E811102C0E12CF12C8091010100E06A
:1005000010E0882309F489C030E83F838FE38D83AE
:1005100049C081E0881682E098060CF076C000E0C1
:1005200010E021E0C21622E0D2060CF0A1CF30E8A4
:100530003F838FE38D8320C000E010E0341098CF1C
:1005400020E82F833FE33D8317C09B01AC01B80136
:100550008F819D810E94DC0418160CF456C0930113
:10056000A701B8018F819D810E947D0300E010E00A
:1005700087FD4EC01F821D82612C712CE12CF12C55
:1005800011C09301A701B8018F819D810E94DC04F5
:1005900087FD08C03801EF80FD800A811B813C8106
:1005A0003F835D8220E030E04FE753E4B301C701B1
:1005B0000E94E10420E030E040E05FE30E9411038C
:1005C0000E94F403F62E862F972F90938B00809332
:1005D0008A0020E030E04FE753E4B8018F819D812D
:1005E0000E94E10420E030E040E05FE30E9411035C
:1005F0000E94F4036093B300F092B400A114B1041C
:1006000009F485CE0E94000082CE00E010E030CFD9
:1006100080E88F832FE32D83AFCF1F821D82C2CF4F
:100620005058BB27AA270E9428030C94A2040E94BA
:10063000940438F00E949B0420F039F49F3F19F491
:1006400026F40C9491040EF4E095E7FB0C948B04D3
:10065000E92F0E94B30458F3BA176207730784079F
:10066000950720F079F4A6F50C94D5040EF4E095E6
:100670000B2EBA2FA02D0B01B90190010C01CA015C
:10068000A0011124FF27591B99F0593F50F4503E07
:1006900068F11A16F040A22F232F342F4427585FF9
:1006A000F3CF469537952795A795F0405395C9F711
:1006B0007EF41F16BA0B620B730B840BBAF09150C9
:1006C000A1F0FF0FBB1F661F771F881FC2F70EC068
:1006D000BA0F621F731F841F48F48795779567953B
:1006E000B795F7959E3F08F0B0CF9395880F08F027
:1006F0009927EE0F9795879508950E94670408F44F
:1007000081E008950E9496030C94A2040E949B0429
:1007100058F00E94940440F029F45F3F29F00C94B3
:100720008B0451110C94D6040C9491040E94B304D0
:1007300068F39923B1F3552391F3951B550BBB2710
:10074000AA2762177307840738F09F5F5F4F220F55
:10075000331F441FAA1FA9F335D00E2E3AF0E0E84C
:1007600032D091505040E695001CCAF72BD0FE2F96
:1007700029D0660F771F881FBB1F2617370748072A
:10078000AB07B0E809F0BB0B802DBF01FF279358E2
:100790005F4F3AF09E3F510578F00C948B040C9417
:1007A000D6045F3FE4F3983ED4F38695779567953A
:1007B000B795F7959F5FC9F7880F911D9695879517
:1007C00097F90895E1E0660F771F881FBB1F621736
:1007D00073078407BA0720F0621B730B840BBA0BF4
:1007E000EE1F88F7E09508950E94FB036894B1110D
:1007F0000C94D60408950E94BB0488F09F5798F08B
:10080000B92F9927B751B0F0E1F0660F771F881F15
:10081000991F1AF0BA95C9F714C0B13091F00E942F
:10082000D504B1E008950C94D504672F782F88275C
:10083000B85F39F0B93FCCF3869577956795B39556
:10084000D9F73EF490958095709561957F4F8F4FC5
:100850009F4F0895E89409C097FB3EF490958095CA
:10086000709561957F4F8F4F9F4F9923A9F0F92F76
:1008700096E9BB279395F695879577956795B795F4
:10088000F111F8CFFAF4BB0F11F460FF1BC06F5FDA
:100890007F4F8F4F9F4F16C0882311F096E911C0EC
:1008A000772321F09EE8872F762F05C0662371F00D
:1008B00096E8862F70E060E02AF09A95660F771F21
:1008C000881FDAF7880F9695879597F90895990FFD
:1008D0000008550FAA0BE0E8FEEF16161706E8070A
:1008E000F907C0F012161306E407F50798F0621B2B
:1008F000730B840B950B39F40A2661F0232B242B00
:10090000252B21F408950A2609F4A140A6958FEF1E
:10091000811D811D089597F99F6780E870E060E070
:1009200008959FEF80EC089500240A941616170688
:1009300018060906089500240A94121613061406D0
:1009400005060895092E0394000C11F4882352F033
:10095000BB0F40F4BF2B11F460FF04C06F5F7F4FEB
:100960008F4F9F4F089557FD9058440F551F59F0D2
:100970005F3F71F04795880F97FB991F61F09F3F8C
:1009800079F087950895121613061406551FF2CFB5
:100990004695F1DF08C0161617061806991FF1CF05
:1009A00086957105610508940895E894BB2766272C
:1009B0007727CB0197F908950E94670408F48FEF19
:1009C00008950E94F4040C94A2040E94940438F048
:1009D0000E949B0420F0952311F00C948B040C943E
:1009E000910411240C94D6040E94B30470F3959FD3
:1009F000C1F3950F50E0551F629FF001729FBB2716
:100A0000F00DB11D639FAA27F00DB11DAA1F649FB1
:100A10006627B00DA11D661F829F2227B00DA11D64
:100A2000621F739FB00DA11D621F839FA00D611DEA
:100A3000221F749F3327A00D611D231F849F600D0B
:100A4000211D822F762F6A2F11249F5750409AF034
:100A5000F1F088234AF0EE0FFF1FBB1F661F771FC0
:100A6000881F91505040A9F79E3F510580F00C948B
:100A70008B040C94D6045F3FE4F3983ED4F3869540
:100A800077956795B795F795E7959F5FC1F7FE2B2B
:100A9000880F911D9695879597F90895F894FFCF43
:00000001FF
